:10000000A728FF3FFF3FFF3FA53003138312DA000D
:10001000DA0B082800000000080003138312A50172
:10002000210884000008D3000130D1002208D2004A
:100030005108D000520803192128D00D5010FF3F5D
:100040001B285308D0055008D100520803192C284A
:10005000D10CD113FF3F262851082406031D5A282E
:100060002308003C0318382804200420A303302868
:10007000210884000008D3000130D1002208D200FA
:100080005108D000520803194928D00D5010FF3FE5
:1000900043285308D0055008D100520803195428AA
:1000A000D10CD113FF3F4E2851082406031D5A28B6
:1000B000FF30A5002508D000080003138312851621
:1000C0001A30DB00FF30DA00DB0B67286A28DA0B16
:1000D00067286428E730DA00DA0B6C280000051581
:1000E0001A30DB00FF30DA00DB0B77287A28DA0BD6
:1000F00077287428E730DA00DA0B7C2800008514B2
:100100000514080003138312051085101A30DB0054
:10011000FF30DA00DB0B8D289028DA0B8D288A2837
:10012000E730DA00DA0B9228000005111A30DB0004
:10013000FF30DA00DB0B9D28A028DA0B9D289A28D7
:10014000E730DA00DA0BA228000085120800073039
:1001500003138312990083169F011830850018300D
:10016000831285000530A1000430A2006430A30092
:10017000A4010D205008FF3A031DCB285D2000305C
:10018000051A0130D1005108003A031DC9280000AA
:10019000BF288220B2280530A1000330A20005301C
:1001A000A300A4010D205008FF3A031D07295D207C
:1001B000003085190130D1005108003A031DE228B2
:1001C0000000D828A001A0012008FF3C031C05293D
:1001D0000430DB00FF30DA00DB0BEF28F228DA0B0B
:1001E000EF28EC28E230DA00DA0BF4280030851929
:1001F0000130D1005108003A031DFF28D8282008FB
:10020000FF3A03190529A00AE4288220CB28B22846
:100210000829FF3FFF3FFF3FFF3FFF3FFF3FFF3FFB
:02400E00543F1D
:00000001FF
